:1000000000308A009D280000D3346D38EC32202A5D
:10001000E832F236EF36653AE832F2060A00A831E5
:100020002910CB306B36E9352019B018B3060A0019
:10003000F73B77176D366131AE31FA060A00831649
:100040008613831286130830F80026280000F8175C
:100050003728F813A40C03188617031C8613781787
:1000600037287813F80B2A283528000086173F30E8
:100070008400840B39280000F81B2928781B3128BC
:100080000800831603178C170C140000000083125D
:100090000C087F39031985280313A10003170D08E5
:1000A0000313A20003170F080313A3002108A400E1
:1000B0001F20220803178D000313230803178F0046
:1000C00083168C170C140000000083120C0D0E0D0B
:1000D0007F39031985280313A10003170D080313A3
:1000E000A20003170F080313A3002108A4001F2078
:1000F000220803178D000313230803178F008D0AAE
:1001000003198F0A03134128031703130800213032
:1001100084008313000803199A280230F800F701BD
:10012000F70B9028F80B8F289730F700F70B9628DD
:10013000800B8D288A110A121629840183131F301F
:100140008305713083168F000F088613831286177C
:10015000831603170908C039890003131F129F1261
:100160000030031788008312870188018901FF305E
:100170000313A000831603170908C039890003136D
:100180001F129F12003003178800831203131F13DE
:100190009F1383169F1383121F149412A01220081A
:1001A0008316870083122016200883168700831287
:1001B000A0112008831687000130831294000030BC
:1001C000831694000108C739083881008312900112
:1001D0000030F80092000030831692008312201540
:1001E0002008831687008312970183169B019C01C8
:1001F00001309D00831203178701880189010430B3
:100200008D0000308F00031341200F3003178D0045
:1002100000308F0003134120183003178D00003089
:100220008F00031341206430A10087281329630045
:04400E00F52CFF3F4F
:00000001FF
